:100000000C94E5010C9402020C9402020C9402027E
:100010000C9402020C9402020C9402020C94020250
:100020000C9402020C9402020C9402020C94020240
:100030000C9402020C9402020C94E7060C94020247
:100040000C9402020C948E030C9431030C94F30272
:100050000C9402020C94FA080C9402020C94020212
:100060000C9402020C940202901C931CA21CDB1C38
:10007000ED1C0A1D1C1D341D891D08215D1F621FFA
:100080001120432074209020B020E82008214261F4
:10009000756472617465206F666620627920256CD4
:1000A000646270730A00756E6974203C2053455277
:1000B0005F434E5400626572746F732F6370752FC7
:1000C0006176722F6472762F7365725F6D656761FA
:1000D0002E630073697A65203E2031006265727478
:1000E0006F732F7374727563742F6669666F6275B0
:1000F000662E680066642D3E68772D3E72786275C4
:100100006666657200626572746F732F6472762F13
:100110007365722E630066642D3E68772D3E747899
:1001200062756666657200626572746F732F6472C1
:10013000762F7365722E63002166642D3E69735FAE
:100140006F70656E00626572746F732F6472762FC4
:100150007365722E6300756E6974203C20636F7541
:100160006E746F66287365725F68616E646C657328
:100170002900626572746F732F6472762F736572D3
:100180002E6300706F72742D3E69735F6F70656EC1
:1001900000626572746F732F6472762F7365722EAE
:1001A000630066642D3E5F74797065203D3D204B91
:1001B00046545F53455249414C00626572746F73F7
:1001C0002F6472762F7365722E68002174696D65D5
:1001D000725F696E697469616C697A6564006265F1
:1001E00072746F732F6472762F74696D65722E63EB
:1001F000002674696D65722D3E6C696E6B006265D8
:1002000072746F732F6472762F74696D65722E63CA
:100210000066642D3E7265616400626572746F737E
:100220002F696F2F6B66696C652E680066642D3EC2
:10023000777269746500626572746F732F696F2FCE
:100240006B66696C652E68006368203C3D20350054
:100250004D6F64656D2F68617264776172652E639E
:100260000066642D3E5F74797065203D3D204B46ED
:10027000545F4146534B004D6F64656D2F6166734B
:100280006B2E6800808183848687898A8C8E8F910B
:1002900092949597989A9B9D9EA0A2A3A5A6A7A984
:1002A000AAACADAFB0B2B3B5B6B7B9BABCBDBEC0FB
:1002B000C1C2C4C5C6C8C9CACBCDCECFD0D2D3D493
:1002C000D5D6D7D9DADBDCDDDEDFE0E1E2E3E4E559
:1002D000E6E7E8E9EAEAEBECEDEEEEEFF0F1F1F259
:1002E000F3F3F4F5F5F6F6F7F8F8F9F9FAFAFAFB9C
:1002F000FBFCFCFCFDFDFDFDFEFEFEFEFEFFFFFF28
:10030000FFFFFFFF66642D3E636C6561726572726C
:1003100000626572746F732F696F2F6B66696C650D
:100320002E680066642D3E6572726F72006265729F
:10033000746F732F696F2F6B66696C652E6800632D
:100340006F756E74203C3D2038004D6F64656D2FD5
:10035000636F6D7072657373696F6E2F686561741A
:10036000736872696E6B5F656E636F6465722E632E
:10037000006275665F706F696E746572203E3D2025
:1003800062756600626572746F732F6D7761726556
:100390002F666F726D617477722E6300203D20307E
:1003A0007825700A00496E76616C696420707472F9
:1003B0003A20003A2000417373657274696F6E20B1
:1003C0006661696C65643A20000011241FBECFEF9E
:1003D000D8E0DEBFCDBF11E0A0E0B1E0E4E0FDE594
:1003E00002C005900D92A436B107D9F716E0A4E635
:1003F000B1E001C01D92AF31B107E1F70E942208C0
:100400000C94802E0C9400001092C00088E9809318
:10041000C10008951092C1000895FC0122852111A8
:1004200005C021E0228788EB8093C1000895E2ECAB
:10043000F0E0808194E0660F771F9A95E1F78F7C5A
:10044000862B808308959FB7F89484B1886284B91D
:100450009FBF8FB7F894229A8FBF8FB7F8942498D4
:100460008FBF80ED8CBD8CB581608CBD8DB58E7FCE
:100470008DBD08951CBC9FB7F89484B1837C84B96A
:100480009FBF089508950895FC01828508956FB770
:10049000F894DC011A962C911A97211120C0E09152
:1004A0001206F0911306478D50A121A132A14217E7
:1004B0005307A9F021E01A962C93A78DB0A185A12E
:1004C00096A1A817B90719F483A194A104C0A78D18
:1004D000B0A1CD01019690A3878F8C918EBD6FBF87
:1004E00008954F925F926F927F928F929F92AF92F8
:1004F000BF92CF92DF92EF92FF92CF93DF934A01A8
:100500005B01CB01BA019695879577956795605CFD
:100510007D4B804F9F4FA50194010E94702CE901F3
:1005200021974427552760E472E48FE090E00E9411
:10053000382C75016401C61AD70AE80AF90A26019F
:100540003701F7FE07C04424552432014C185D08DA
:100550006E087F08C501B40121E230E040E050E0C0
:100560000E94702C241535054605570580F4FF922E
:10057000EF92DF92CF928EE890E09F938F930E944C
:1005800060290F900F900F900F900F900F90D093C5
:10059000C500C093C400DF91CF91FF90EF90DF9032
:1005A000CF90BF90AF909F908F907F906F905F9013
:1005B0004F900895CF93DF93EC018230910544F082
:1005C0004AE953E065EB70E086EA90E00E94E22998
:1005D0002BE02C9FC0012D9F900D1124865F9E4F14
:1005E000DF91CF9108951F920F920FB60F921124B1
:1005F0002F933F938F939F93AF93BF93EF93FF936B
:10060000E0911006F0911106278D30A181A192A1F1
:100610002817390731F488E98093C100109214013A
:1006200013C0A78DB0A185A196A1A817B90719F489
:1006300083A194A104C0A78DB0A1CD01019690A380
:10064000878F8C918093C600FF91EF91BF91AF91FE
:100650009F918F913F912F910F900FBE0F901F9000
:1006600018951F920F920FB60F9211242F933F935C
:100670004F935F938F939F93AF93BF93EF93FF93AA
:10068000E0911006F091110697A58091C000887145
:10069000892B87A75091C60027A130A583A594A5D3
:1006A0002817390739F421A532A585A596A528175D
:1006B000390761F021A532A587A190A5019741E0F6
:1006C0002817390709F040E0842F01C081E080FF3E
:1006D00004C087A5816087A712C0A1A5B2A55C93BD
:1006E00021A532A585A596A52817390719F483A554
:1006F00094A503C081A592A5019692A781A7FF9119
:10070000EF91BF91AF919F918F915F914F913F91E9
:100710002F910F900FBE0F901F9018951F920F9260
:100720000FB60F9211242F933F934F938F939F9364
:10073000AF93BF93EF93FF93E0911206F0911306EE
:1007400027A130A583A594A52817390739F421A539
:1007500032A585A596A52817390761F021A532A5F0
:1007600087A190A5019741E02817390709F040E0DB
:10077000842F01C081E080FD13C08EB5A1A5B2A574
:100780008C9321A532A585A596A52817390719F4BC
:1007900083A594A503C081A592A5019692A781A7E0
:1007A000E0911206F0911306278D30A181A192A14C
:1007B0002817390799F0A78DB0A185A196A1A81790
:1007C000B90719F483A194A104C0A78DB0A1CD01EC
:1007D000019690A3878F8C918EBD02C010921F014D
:1007E000FF91EF91BF91AF919F918F914F913F9169
:1007F0002F910F900FBE0F901F9018959FB7F894F0
:1008000083E085BB14BC15BC82E084BD85B58360E4
:1008100085BD16BC89EF87BDEEE6F0E080818E7F56
:1008200080838081826080839FBF0895CF93DF9310
:10083000EC01FB015FB7F894278D30A183A194A14F
:1008400028173907E9F421A132A185A196A128171B
:100850003907B1F481E05FBF80FD11C04FB7F89454
:10086000A1A1B2A1CC9321A132A185A196A1281763
:10087000390799F483A194A192A381A314C0DACF7C
:1008800081A192A1278D30A12150310941E0821729
:10089000930709F040E0842FDECF21A132A12F5F22
:1008A0003F4F32A321A34FBF80A991A9DC01ED9155
:1008B000FC910084F185E02D0995CE019927DF9107
:1008C000CF910895FC014FB7F89427A130A581A5D9
:1008D00092A54FBF2817390739F087A5897B79F092
:1008E00024C087A5897BC9F74FB7F89427A130A505
:1008F00081A592A54FBF2817390799F3EECF2FB7DF
:10090000F894A7A1B0A585A596A5A817B90719F4CD
:1009100083A594A504C0A7A1B0A5CD01019690A779
:1009200087A38C912FBF90E008958FEF9FEF0895DC
:10093000AF92BF92CF92DF92EF92FF920F931F93ED
:10094000CF93DF937C015B016A01FC01008911896F
:10095000228933890C3412452544334541F04CEB50
:1009600050E06AEB71E082EA91E00E94E229E50141
:1009700000E010E00C151D0559F0C7010E9462044B
:100980008F3F2FEF920721F00F5F1F4F8993F2CF18
:10099000C801DF91CF911F910F91FF90EF90DF90F1
:1009A000CF90BF90AF900895AF92BF92CF92DF9259
:1009B000EF92FF920F931F93CF93DF937C015B0124
:1009C0006A01FC0100891189228933890C3412459E
:1009D0002544334541F04CEB50E06AEB71E082EA8C
:1009E00091E00E94E229E50100E010E00C151D05F0
:1009F00061F08991B701992787FD90950E941604AF
:100A0000019619F00F5F1F4FF1CFC801DF91CF9111
:100A10001F910F91FF90EF90DF90CF90BF90AF901C
:100A20000895CF93DF93EC01488959896A897B89BE
:100A30004C3452456544734541F04CEB50E06AEB51
:100A400071E082EA91E00E94E2298FA590E0DF91B7
:100A5000CF910895CF93DF93EC01488959896A8932
:100A60007B894C3452456544734541F04CEB50E072
:100A70006AEB71E082EA91E00E94E2291FA6DF9111
:100A8000CF910895CF93DF93EC01488959896A8902
:100A90007B894C3452456544734549F04CEB50E03A
:100AA0006AEB71E082EA91E00E94E22900C02F8D9A
:100AB00038A189A19AA128173907C9F788A999A946
:100AC000DC01ED91FC910284F385E02D0995811103
:100AD000EECF80E090E0DF91CF910895EF92FF920A
:100AE0000F931F93CF93DF93EC018B01623071055D
:100AF00040F042E651E062E771E086E591E00E9455
:100B0000E229F801EE0FFF1FE05FF94FD183C083A8
:100B10008E8D882341F045E651E065E471E088E37D
:100B200091E00E94E22981E08E8F1D8F0C8FC80119
:100B30000E94DA0299AB88ABDC0112968D919C91F0
:100B40001397892B41F44DE651E067E271E086E1AD
:100B500091E00E94E229E8A9F9A984819581892B75
:100B600041F44EE651E065E071E084EF90E00E94D0
:100B7000E229E8A9F9A9E680F78002811381B2E0B1
:100B8000EB16F10440F441E251E06CED70E083EDCE
:100B900090E00E94E2291CA30BA31AA309A318A3A7
:100BA0000F8FC7010197800F911F9EA38DA3E8A906
:100BB000F9A9E084F18404811581E2E0EE16F104E4
:100BC00040F441E251E06CED70E083ED90E00E9472
:100BD000E2291CA70BA71AA709A718A70FA3C701EB
:100BE0000197800F911F9EA78DA788A999A9DC0165
:100BF000ED91FC910190F081E02DBE0109951FA6B9
:100C0000CE01DF91CF911F910F91FF90EF9008954A
:100C1000FC014FB7F89427A130A581A592A54FBF3D
:100C200028173907B1F02FB7F894A7A1B0A585A56B
:100C300096A5A817B90719F483A594A504C0A7A180
:100C4000B0A5CD01019690A787A38C912FBF90E00E
:100C500008958FEF9FEF08956FB7F894FC0147A1B7
:100C600050A521A532A56FBF81E04217530709F4B3
:100C700080E00895DC01D0968D919C91D197DC01A4
:100C8000ED91FC910480F581E02D09944FB7F89423
:100C9000FC0121A532A530A727A34FBF08954FB768
:100CA000F894FC0121A132A130A3278F4FBF0895F2
:100CB000CF93DF93EC010E944606CE01DF91CF91E6
:100CC0000C944F06CF93DF93EC01488959896A89C8
:100CD0007B894C3452456544734541F04CEB50E000
:100CE0006AEB71E082EA91E00E94E2298E8D811127
:100CF00008C04BE851E061E971E083E891E00E94AF
:100D0000E2291E8ECE010E94420588A999A9DC0124
:100D1000ED91FC910280F381E02D099519AA18AAA2
:100D2000CE010E94580680E090E0DF91CF910895B7
:100D3000CF93DF93EC01488959896A897B894C34C8
:100D400052456544734541F04CEB50E06AEB71E06D
:100D500082EA91E00E94E229CE010E9462066C8D37
:100D60007D8DCE010E946E05CE01DF91CF91089559
:100D7000FC01CB0122E3DF011D922A95E9F74CE447
:100D800052E565E473E5408B518B628B738B28E9E8
:100D900036E03583248322E636E03783268328E94C
:100DA00034E03183208324ED34E03383228322E452
:100DB00035E03387228721E135E0358724872AE231
:100DC00035E037872687BC01CF010C946E051F9252
:100DD0000F920FB60F9211240F931F932F933F93EF
:100DE0004F935F936F937F938F939F93AF93BF9333
:100DF000CF93DF93EF93FF938091140690911506A4
:100E0000A0911606B09117060196A11DB11D809301
:100E1000140690931506A0931606B09317060BEAD6
:100E20001AEBC091A401D091A50188819981892BE9
:100E3000D1F18FB7F8944091140650911506609146
:100E40001606709117068FBF88859985AA85BB8580
:100E5000481B590B6A0B7B0B77FD25C0CF3FD10593
:100E600009F048F42BEC30E04EEF51E061EF71E017
:100E7000CE010E94F829EA81FB81888199819183C2
:100E80008083E881F9818A819B81938382831B829D
:100E90001A82198218821B8B0A8BEC85FD85CE0184
:100EA0000C960995BECFFF91EF91DF91CF91BF9145
:100EB000AF919F918F917F916F915F914F913F91F2
:100EC0002F911F910F910F900FBE0F901F901895AB
:100ED00088EA91E09093A5018093A4011092A70164
:100EE0001092A6011092A9011092A80184EA91E043
:100EF0009093AB018093AA011092140610921506EC
:100F000010921606109217060E94FE038091180692
:100F1000882341F041E951E06EED71E08BEC91E006
:100F20000E94E22981E0809318060895EF92FF92D3
:100F30000F931F93CF93DF931F92CDB7DEB77C0142
:100F40008B018983DB0112968D919C911397892BDC
:100F500041F44EE051E066E372E08CE292E00E94E0
:100F6000E229D8011296ED91FC91139741E050E0EF
:100F7000BE016F5F7F4FC8010995019719F4C70142
:100F8000992702C08FEF9FEF0F90DF91CF911F91B4
:100F90000F91FF90EF9008950F931F93CF93DF93DE
:100FA0001F92CDB7DEB78C01DC018D919C91892B0E
:100FB00041F442EF50E06AE172E081E192E00E9488
:100FC000E229D801ED91FC9141E050E0BE016F5F54
:100FD0007F4FC8010995019719F4898190E002C0FB
:100FE0008FEF9FEF0F90DF91CF911F910F91089599
:100FF000CF92DF92EF92FF92CF93DF93EC01C12C5F
:10100000D12C76014A815B8160E070E0C416D50680
:10101000E606F70680F4E881F981EC0DFD1D80817C
:1010200067EB72E090E00E9496078FEFC81AD80A2B
:10103000E80AF80AE7CFDF91CF91FF90EF90DF90B9
:10104000CF90089578940E94680760E070E087EB85
:1010500092E00E94B80640E855E260E070E087EB5D
:1010600092E00E943A0686E08093C20060E070E061
:101070008CE294E00E94A50D48EF57E06CE274E02A
:1010800089EE92E00E947F0F8FB7F894C09014060B
:10109000D0901506E0901606F09017068FBFC1E0BD
:1010A00089EE92E00E9424198091AC0181112EC03A
:1010B00087EB92E00E942C06882341F187EB92E0B7
:1010C0000E9408068093AF019093B0012091AD017A
:1010D0003091AE01F901EF54FE4FA9014F5F5F4F10
:1010E00080835093AE014093AD012530314010F024
:1010F000C093AC018FB7F894C0901406D090150639
:10110000E0901606F09017068FBF1BC08091AD01CE
:101110009091AE01892BA9F02FB7F8948091140615
:1011200090911506A0911606B09117062FBF8C1945
:101130009D09AE09BF090397A105B10514F0C0933D
:10114000AC018091AC01882309F4AACF89EE92E02A
:101150000E94280F8111A4CF4091AD015091AE01A2
:1011600061EB71E089EE92E00E94C3141092AC0131
:101170001092AE011092AD0193CFCF93DF93EC01AB
:1011800070930705609306058630910544F041E2AF
:1011900050E060E572E088E492E00E94E22910925B
:1011A000800089E18093810082E896E09093870037
:1011B000809386008C2F806480937C0087B121E02F
:1011C00030E001C0220FCA95EAF7922F909589234B
:1011D00087B988B1892388B980917E00822B80935A
:1011E0007E0087E080937B008CEE80937A00DF9115
:1011F000CF9108951F920F920FB60F9211242F9343
:101200003F934F935F936F937F938F939F93AF938E
:10121000BF93EF93FF9380E286BB6091780070915B
:101220007900769567957695679560588091060563
:10123000909107050E94BC0A80911A06882349F004
:1012400080910605909107050E948C0C807F886034
:1012500007C080911906882311F088E801C080E852
:101260008BB9FF91EF91BF91AF919F918F917F913A
:101270006F915F914F913F912F910F900FBE0F9003
:101280001F901895AF92BF92CF92DF92EF92FF928C
:101290000F931F93CF93DF936C01EB017A01DC0175
:1012A00050960D911D912D913C9153970D341B44F7
:1012B0002345364441F04EE650E067E772E081E6B0
:1012C00092E00E94E2295E01CE018E0D9F1DF60183
:1012D000EB57FF4FA816B90671F4C5018C1B9D0B87
:1012E000DF91CF911F910F91FF90EF90DF90CF9002
:1012F000BF90AF9008956FB7F894408151812281DB
:1013000033816FBF4217530741F32FB7F894C09052
:101310001406D0901506E0901606F09017062FBF21
:101320006FB7F89440815181228133816FBF42179A
:101330005307A9F44FB7F8940091140610911506BD
:1013400020911606309117064FBF0C191D092E0962
:101350003F09101611061206130614F7BECF6FB719
:10136000F89420813181468157812417350719F47B
:101370004481558105C020813181A9014F5F5F4FB4
:1013800051834083D9012C916FBFD5012D935D010D
:10139000A1CF6F927F928F929F92AF92BF92CF9286
:1013A000DF92EF92FF920F931F93CF93DF93EC01A5
:1013B0008B017A0188899989AA89BB898D349B44DC
:1013C000A345B64441F04EE650E067E772E081E69F
:1013D00092E00E94E229F801A8014E0D5F1D9924B8
:1013E0009394BB24B3943E0187E7680E711C20E4FC
:1013F00030E06CE370E088E0E82EF12CE417F507AC
:1014000009F44EC0AFB6F894CFA4D8A88BA99CA974
:10141000C816D90639F4C9A8DAA88DA99EA9C81694
:10142000D90669F0C9A8DAA88FA598A901978824D8
:101430008394C816D90609F0812C882D01C081E05B
:10144000AFBE80FDDFCFD190AFB6F89489A99AA93D
:10145000DC01DC92C9A8DAA88DA99EA9C816D90614
:1014600019F48BA99CA903C089A99AA901969AABE2
:1014700089ABAFBED3018C9181110CC03EA72DA7C3
:101480001CA61BA61AA69C92299A7BA36AA35B9A08
:10149000B0921A068FB7F894FDA2ECA28FBFAECF20
:1014A000CF01801B910BDF91CF911F910F91FF9086
:1014B000EF90DF90CF90BF90AF909F908F907F90F4
:1014C0006F900895CF93DF93EC01488959896A8919
:1014D0007B894D345B446345764441F04EE650E0F1
:1014E00067E772E081E692E00E94E229C958DF4F87
:1014F00088818111FDCF80E090E0DF91CF91089548
:10150000CF93DF93EC01488959896A897B894D34EF
:101510005B446345764441F04EE650E067E772E095
:1015200081E692E00E94E2292FB7F894C852DF4F7B
:10153000888199812FBFDF91CF910895CF93DF9359
:10154000EC01488959896A897B894D345B4463453C
:10155000764441F04EE650E067E772E081E692E0C3
:101560000E94E2298FB7F894C852DF4F198218827F
:101570008FBFDF91CF910895EF92FF920F931F934A
:10158000CF93DF93FC018C0101531F4FD8014D9184
:101590005C91DC01A353BF4F4D935C93DC01A858D1
:1015A000BF4F8D919C91119716962D913C91179755
:1015B0008217930729F414962D913C91159706C034
:1015C0008D919C9111979C012F5F3F4F11963C93F9
:1015D0002E93EC0128812602900111243595279540
:1015E00035952795E801398328837F01D3EDED0EEA
:1015F000F11CE701888199818F010F521F4FE8018B
:101600009983888395958795840F951F820F931FE3
:10161000E70199838883AF014B525F4F21E0181691
:1016200019060CF020E0EA018881880F822B88835C
:1016300012968D919C911397EC01688312962D91CF
:101640003C91139716968D919C91179728173907FF
:1016500029F414968D919C91159705C012968D9141
:101660009C911397019613969C938E931297DA018F
:101670009C91892F8695869589278370DF01AA52D0
:10168000BF4F833039F48C91803214F48F5F01C0E6
:1016900081508C938C91885F8C9380340CF435C18D
:1016A0008F738C93DF01A952BF4F8C91880F977075
:1016B0002BEF290F233010F0933009F481608C93C5
:1016C0009C91892F8695892780958170968D990F99
:1016D000892B868F8E3709F04EC0DF01AB57BF4F85
:1016E0002D913C91119714968D919C9115972817E7
:1016F000390759F412962D913C91139716968D91B6
:101700009C9117972817390779F012962D913C91E3
:1017100013978D919C911197019741E028173907F4
:1017200009F040E0842F01C081E080FDDDC0129609
:10173000CD91DC9113978EE7888312962D913C9181
:10174000139716968D919C9117972817390729F4AE
:1017500014968D919C91159705C012968D919C9130
:101760001397019613969C938E93129781E081A311
:101770002A9A41E0BCC0982F9F779F3719F411A295
:101780002A98C3C091A1992309F4BFC0982F9F73D1
:101790009E3309F4BAC080FF03C080A1806880A393
:1017A000878D8F5F878F90A1883008F4ACC0DF01F0
:1017B000AB57BF4F82E8890F823018F09B3109F098
:1017C0004BC02D913C91119714968D919C9115973A
:1017D0002817390759F412962D913C9113971696B4
:1017E0008D919C9117972817390779F012962D91B2
:1017F0003C9113978D919C911197019741E0281787
:10180000390709F040E0842F01C081E080FD20C04D
:101810001296CD91DC9113978BE1888312962D91CE
:101820003C91139716968D919C911797281739071D
:1018300029F414968D919C91159705C012968D915F
:101840009C911397019613969C938E93129704C0C4
:1018500011A22A9840E001C041E02D913C911197DE
:1018600014968D919C9115972817390759F4129663
:101870002D913C91139716968D919C91179728174F
:10188000390779F012962D913C9113978D919C9187
:101890001197019751E02817390709F050E0852F7B
:1018A00001C081E080FD20C080A11296CD91DC9125
:1018B0001397888312962D913C91139716968D91CC
:1018C0009C9117972817390729F414968D919C91AC
:1018D000159705C012968D919C91139701961396BA
:1018E0009C938E93129703C011A22A9840E010A2F5
:1018F000178E41110AC0E852FF4F808191818160AB
:101900009183808302C0969590A3DF91CF911F9120
:101910000F91FF90EF900895DC0196968C91969729
:101920008111EAC098968C9198978111A0C09F96DA
:101930002D913C91D097D1968D919C91D29728175B
:10194000390739F494968D919C919597892B09F4D8
:101950005CC099968C919997811103C09A961C92BC
:101960009A9781E099968C93999792968D919C91F4
:101970009397009789F59F962D913C91D097D1969A
:101980008D919C91D2972817390751F494968D9197
:101990009C919597019795969C938E93949721C0CF
:1019A0009F96ED91FC91D097D5968D919C91D6976D
:1019B000E817F90729F4D3968D919C91D49706C026
:1019C0009F96ED91FC91D097CF010196D0969C9374
:1019D0008E939F97808106C0019793969C938E93D8
:1019E00092978EE797968C93979797968C91979767
:1019F0008B3199F59F962D913C91D097D1968D91F1
:101A00009C91D2972817390749F45B9810921A06CF
:101A1000A958BF4F1C92299880E008959F96ED9198
:101A2000FC91D097D5968D919C91D697E817F907A0
:101A300029F4D3968D919C91D49706C09F96ED91F1
:101A4000FC91D097CF010196D0969C938E939F974F
:101A5000808197968C93979706C08E57823018F4A2
:101A600099961C92999781E098968C93989799965D
:101A70002C9199979D968D919C919E972223A9F0E8
:101A80009A962C919A97253080F09A961C929A9764
:101A90008034910519F485E790E002C080E490E07D
:101AA0009E969C938E939D9723C098963C91989771
:101AB00097962C919797232341F09A968C919A9719
:101AC0008F5F9A968C939A970FC09A961C929A97CA
:101AD0008034910519F485E790E002C080E490E03D
:101AE0009E969C938E939D97330F98963C939897D0
:101AF00088E096968C9396979D96ED91FC919E9793
:101B00009B968D919C919C97E80FF91F9F013170D6
:101B10009C963C932E939B9796968C91969781508A
:101B200096968C93FF27E038F10530F08FEF90E028
:101B3000AC014E1B5F0BFA01EC57FD4F84912F3F18
:101B4000310511F008F080950895CF93DF93EC01F3
:101B5000CB012AEDFE0111922A95E9F77D8F6C8F5A
:101B600020E430E03EA72DA79E0120583F4FFE0104
:101B7000E858FF4F358324833383228331832083C6
:101B80009E012C573F4F378326839E0123573F4F9B
:101B9000DE01AB57BF4F15963C932E9314971396C7
:101BA0003C932E93129711963C932E939E012453AF
:101BB0003F4F17963C932E9316979E01295C3F4FFB
:101BC0003CAB2BAB3AAB29AB38AB2FA79E012A58C5
:101BD0003F4F3EAB2DAB24E030E0A281B3811C929D
:101BE00062817381468157816417750719F44481B6
:101BF000558104C0428153814F5F5F4F53834283BD
:101C0000215031092115310541F7BE010E94BD085F
:101C10008AB1886F8AB9219A229A4DE45BE463E520
:101C200076E4488B598B6A8B7B8B89EC99E09B839C
:101C30008A8382E499E09983888382E69AE09B878D
:101C40008A8780E89AE09D878C878EE99AE09F8753
:101C50008E87DF91CF9108952F923F924F925F929E
:101C60006F927F928F929F92AF92BF92CF92DF92AC
:101C7000EF92FF920F931F93CF93DF93CDB7DEB711
:101C800028970FB6F894DEBF0FBECDBF282F217066
:101C90002B8383FB442440F8512C81FBAA27A0F915
:101CA000B0E0A425B52584FB332730F93F8318869F
:101CB00086FB772770F979831A8282FB662460F8A5
:101CC000712C85FB222420F8312C8078E82FF0E05D
:101CD000EE0FEF2FEE1FFF0BFE83ED83F62FF1705B
:101CE000FC8363FB882480F8912C61FB222720F978
:101CF00030E02825392564FB442740F950E066FB95
:101D0000002700F910E062FBCC24C0F8D12C65FB61
:101D1000EE24E0F8F12C607870E0660F672F661F04
:101D2000770B402751275A01AE24BF24A626B72699
:101D3000C9018C259D258627972736E0880F991F96
:101D40003A95E1F760E8A69E80191124EF81F885A5
:101D500069817A81E627F727F887EF839E2F9170B4
:101D60007B8197273A2F31709327890FA625B725B6
:101D7000ED81FE81AE27BF27F4E0AF9F800D1124D7
:101D8000EF81F885E225F3256D817E81E627F7272F
:101D900078E0E79F800D112441709C8149272170D4
:101DA0004227E0E14E9F800D112496012E253F250C
:101DB000922F9170FC819F2708251925017090278B
:101DC00020E2929F800D1124930122253325922F2A
:101DD00091703B81932729813A81242535252170F3
:101DE000922762E0969F800D112428960FB6F894F2
:101DF000DEBF0FBECDBFDF91CF911F910F91FF903E
:101E0000EF90DF90CF90BF90AF909F908F907F909A
:101E10006F905F904F903F902F9008951F93CF93B6
:101E2000DF93EC01162F82E8860F823010F06B31C1
:101E300031F4688179818BE190E00E949607688196
:101E40007981812F90E0DF91CF911F910C949607BB
:101E50000F931F93CF93DF93EC01FC01EE5BFE4FDA
:101E6000808181110FC02FB7F89480911406909152
:101E70001506A0911606B09117062FBF808390E03B
:101E80000E942C2E8FB7F89440911406509115069D
:101E900060911606709117068FBFCF5DDE4F0881E7
:101EA00019812A813B81401B510B620B730B403B14
:101EB000510561057105DCF00E94272E6FEF70E07F
:101EC0000E945C2C8535A8F08FB7F89440911406D9
:101ED0005091150660911606709117068FBF4B54EE
:101EE000510961097109488359836A837B8381E0C1
:101EF00001C080E0DF91CF911F910F91089523E4FD
:101F000031E0DC01F9011D923197E9F7FC01EC5E4B
:101F1000FE4F71836083FC01E55EFE4F5183408379
:101F20002FB7F8944091140650911506609116064B
:101F3000709117062FBFFC01EF5DFE4F4083518368
:101F400062837383FC01EE5BFE4F10820895CF9293
:101F5000DF92EF92FF920F931F93CF93DF9300D006
:101F600000D0CDB7DEB76C017B0164E088E00E9451
:101F7000901E8C01009749F11C821B821A821982E3
:101F80009E012F5F3F4FA701B6010E94C11EC801ED
:101F90000E94392129813A812E153F0520F4C8017C
:101FA0000E946D1E12C0019751F49E012D5F3F4F9C
:101FB00048E051E068E075E0C8010E94131FC801C5
:101FC0000E946D1E8B819C8102C080E090E00F908A
:101FD0000F900F900F90DF91CF911F910F91FF9075
:101FE000EF90DF90CF900895CF92DF92EF92FF9223
:101FF0000F931F93CF93DF9300D000D0CDB7DEB700
:102000006C017B0144E068E088E091E00E94DC1B09
:102010008C01009749F11C821B821A8219829E0151
:102020002F5F3F4FA701B6010E941B1CC8010E94F1
:10203000B21D29813A812E153F0520F4C8010E9466
:10204000B31B12C0019751F49E012D5F3F4F48E032
:1020500051E068E075E0C8010E945F1CC8010E9461
:10206000B31B8B819C8102C080E090E00F900F90A9
:102070000F900F90DF91CF911F910F91FF90EF90F4
:10208000DF90CF9008952F923F924F925F926F9280
:102090007F928F929F92AF92BF92CF92DF92EF92F8
:1020A000FF920F931F93CF93DF93CDB7DEB72A979D
:1020B0000FB6F894DEBF0FBECDBF4C01FC01E75D4B
:1020C000FE4F8081D401A80FB11DA65DBE4F6C9359
:1020D0008F5F80838C3009F01DC494012C5E3E4FCD
:1020E0003A8729879401265D3E4F3A832983D90197
:1020F0004C91407881E090E0403811F080E090E031
:102100009695982F8827979587955401B5EDAB1A2A
:10211000BEEFBB0AF5014081407851E0403809F03C
:1021200050E0682FF0E45F9F600D112464012CECF7
:10213000C21A2EEFD20AD6019C91907841E09038D5
:1021400009F040E0640F7401B3EDEB1ABEEFFB0A37
:10215000F7019081907841E0903809F040E0F0E29A
:102160004F9F600D11248401025D1E4FD8019C9188
:10217000907841E0903809F040E0B0E14B9F600D6D
:1021800011243401E0ED6E1AEEEF7E0AD3019C912A
:10219000907841E0903809F040E0B8E04B9F600D46
:1021A00011242401EFEC4E1AEEEF5E0AD2019C914D
:1021B000907841E0903809F040E0B4E04B9F600D2A
:1021C00011241401EDEC2E1AEEEF3E0AD1014C91D0
:1021D000407881E090E0403811F080E090E0880F96
:1021E000991F680F89859A850E940E0FE981FA81EF
:1021F000408181E090E046FD02C080E090E096954D
:10220000982F882797958795D5015C9141E056FFD7
:1022100040E0682FB0E44B9F600D1124F6018081EF
:1022200091E086FF90E0690FD7018C9191E086FFE5
:1022300090E0B0E29B9F600D1124F801808191E055
:1022400086FF90E0F0E19F9F600D1124D3018C91F7
:1022500091E086FF90E0B8E09B9F600D1124F201B1
:10226000808191E086FF90E0F4E09F9F600D112453
:10227000D1014C9181E090E046FD02C080E090E009
:10228000880F991F680F89859A850E940E0FE98132
:10229000FA81408181E090E045FD02C080E090E05D
:1022A0009695982F882797958795D5015C9141E061
:1022B00055FF40E0682FB0E44B9F600D1124F601FC
:1022C000808191E085FF90E0690FD7018C9191E0CA
:1022D00085FF90E0B0E29B9F600D1124F8018081A2
:1022E00091E085FF90E0F0E19F9F600D1124D30104
:1022F0008C9191E085FF90E0B8E09B9F600D1124E8
:10230000F201808191E085FF90E0F4E09F9F600DF5
:102310001124D1014C9181E090E045FD02C080E0A4
:1023200090E0880F991F680F89859A850E940E0F8B
:10233000E981FA81408181E090E044FD02C080E0C3
:1023400090E09695982F882797958795D5015C9171
:1023500041E054FF40E0682FB0E44B9F600D112432
:10236000F601808191E084FF90E0690FD7018C91A4
:1023700091E084FF90E0B0E29B9F600D1124F80192
:10238000808191E084FF90E0F0E19F9F600D112437
:10239000D3018C9191E084FF90E0B8E09B9F600DA9
:1023A0001124F201808191E084FF90E0F4E09F9F8E
:1023B000600D1124D1014C9181E090E044FD02C0F8
:1023C00080E090E0880F991F680F89859A850E94A8
:1023D0000E0F9401265D3E4F3A832983D9014C911B
:1023E00081E090E043FD02C080E090E09695982F58
:1023F0008827979587955401B5EDAB1ABEEFBB0AB8
:10240000F501508141E053FF40E0682FF0E44F9F19
:10241000600D112464012CECC21A2EEFD20AD601F1
:102420008C9191E083FF90E0690F7401B3EDEB1A9A
:10243000BEEFFB0AF701808191E083FF90E0F0E2BC
:102440009F9F600D11248401025D1E4FD8018C9165
:1024500091E083FF90E0B0E19B9F600D1124340177
:10246000E0ED6E1AEEEF7E0AD3018C9191E083FFCE
:1024700090E0B8E09B9F600D11242401EFEC4E1A10
:10248000EEEF5E0AD2018C9191E083FF90E0B4E020
:102490009B9F600D11241401EDEC2E1AEEEF3E0A05
:1024A000D1014C9181E090E043FD02C080E090E0DA
:1024B000880F991F680F89859A850E940E0FE98100
:1024C000FA81408181E090E042FD02C080E090E02E
:1024D0009695982F882797958795D5015C9141E02F
:1024E00052FF40E0682FB0E44B9F600D1124F601CD
:1024F000808191E082FF90E0690FD7018C9191E09B
:1025000082FF90E0B0E29B9F600D1124F801808172
:1025100091E082FF90E0F0E19F9F600D1124D301D4
:102520008C9191E082FF90E0B8E09B9F600D1124B8
:10253000F201808191E082FF90E0F4E09F9F600DC6
:102540001124D1014C9181E090E042FD02C080E075
:1025500090E0880F991F680F89859A850E940E0F59
:10256000E981FA81408181E090E041FD02C080E094
:1025700090E09695982F882797958795D5015C913F
:1025800041E051FF40E0682FB0E44B9F600D112403
:10259000F601808191E081FF90E0690FD7018C9175
:1025A00091E081FF90E0B0E29B9F600D1124F80163
:1025B000808191E081FF90E0F0E19F9F600D112408
:1025C000D3018C9191E081FF90E0B8E09B9F600D7A
:1025D0001124F201808191E081FF90E0F4E09F9F5F
:1025E000600D1124D1014C9181E090E041FD02C0C9
:1025F00080E090E0880F991F680F89859A850E9476
:102600000E0FE981FA8180818170D5019C919170D2
:102610009B831C822B813C8156E0220F331F5A95ED
:10262000E1F73C832B83622F30E8839F60191124EC
:10263000D6018C918170680FF70180818170F0E282
:102640008F9F600D1124D8018C918170B0E18B9F18
:10265000600D1124F30180818170F8E08F9F600D7F
:102660001124D2018C918170B4E08B9F600D1124F4
:10267000F101808181708D831E822D813E81220F28
:10268000331F3E832D83620F89859A850E940E0F2A
:10269000540134EDA31A3EEFB30AD501EC91640165
:1026A000B1EDCB1ABEEFDB0AD6017C917401BEEC12
:1026B000EB1ABEEFFB0AD7015C9184010B5C1E4F45
:1026C000D8014C916E2F607881E090E0603811F075
:1026D00080E090E09695982F88279795879561E000
:1026E000E3FF60E0E82FB0E46B9FE00D11246E2F54
:1026F00091E043FF90E0690F91E0872F8078803868
:1027000009F090E0F0E29F9F600D112491E073FFCB
:1027100090E020E1929F600D112491E0852F807858
:10272000803809F090E038E0939F600D112491E02B
:1027300053FF90E084E0989F600D1124407881E081
:1027400090E0403811F080E090E0880F991F680F0A
:1027500089859A850E940E0FD501EC91D6017C9156
:10276000D7015C91D8014C9181E090E0E6FD02C078
:1027700080E090E09695982F88279795879561E05F
:10278000E2FF60E0E82FB0E46B9FE00D11246E2FB4
:1027900091E042FF90E0690F91E076FF90E0F0E277
:1027A0009F9F600D112491E072FF90E020E1929FC5
:1027B000600D112491E056FF90E038E0939F600D8A
:1027C000112491E052FF90E084E0989F600D112465
:1027D00081E090E046FD02C080E090E0880F991F04
:1027E000680F89859A850E940E0FD501EC91D6015C
:1027F0007C91D7015C91D8014C9181E090E0E5FD9E
:1028000002C080E090E09695982F8827979587954D
:1028100061E0E1FF60E0E82FB0E46B9FE00D112480
:102820006E2F91E041FF90E0690F91E075FF90E01D
:10283000F0E29F9F600D112491E071FF90E020E194
:10284000929F600D112491E055FF90E038E0939F36
:10285000600D112491E051FF90E084E0989F600D9D
:10286000112481E090E045FD02C080E090E0880FF7
:10287000991F680F89859A850E940E0FD5016C916A
:10288000F6017081D7015C91F8014081862F81703B
:10289000F72FF170FF8318862F813885E4E0220F2F
:1028A000331FEA95E1F738872F8330E4839F200DAB
:1028B0001124822F942F9170890F952F9170A4E08D
:1028C0009A9F800D112491E064FF90E0682FB0E89A
:1028D0009B9F6019112491E074FF90E0E0E29E9FBD
:1028E000600D112491E054FF90E0F8E09F9F600D8F
:1028F000112481E090E044FD02C080E090E0880F68
:10290000991F680F89859A850E940E0FF401E75D73
:10291000FE4F10822A960FB6F894DEBF0FBECDBFD1
:10292000DF91CF911F910F91FF90EF90DF90CF90AB
:10293000BF90AF909F908F907F906F905F904F90DF
:102940003F902F9008951F93CF93DF93EC01162FA4
:102950000E94431080910F06882349F0612F8091D7
:102960000E060E942C0E682FCE010E944310109379
:102970000E0680910F0691E0892780930F06DF9164
:10298000CF911F9108955F926F927F928F929F9245
:10299000AF92BF92CF92DF92EF92FF920F931F936D
:1029A000CF93DF93EC015B017A0110920F0681E077
:1029B000809319068FB7F89440911406509115062C
:1029C00060911606709117068FBF8FB7F89400912B
:1029D00014061091150620911606309117068FBF28
:1029E000041B150B260B370B37FDEFCF8E01025E54
:1029F0001E4F8AEAD8018C93FE01E75DFE4F1082DC
:102A0000B701C5010E94A70F6C01009769F08E15F0
:102A10009F0550F4AC0168E075E0C5010E94372EB7
:102A200076019924939401C0912C6E01BCEECB1ACF
:102A3000BEEFDB0AF601608171818EE790E00E94B3
:102A40009607911002C060E001C062E082E08E0D46
:102A5000877031F198E0981B892E912C6160C40138
:102A6000F4E0880F991FFA95E1F76827D8018C9157
:102A700086278C93CE010E94A314612C712CA5E5AE
:102A80005A2EF80180818525808365E5CE010E945C
:102A9000A314FFEF6F1A7F0A6814790494F307C038
:102AA000D8018C9186278C93CE010E94A3144501F6
:102AB000EA0CFB1C8E149F0469F0F401D4018D9183
:102AC0004D01D8019C9189278C936081CE010E9491
:102AD000A314F0CFF8016081CE010E94A314D601A7
:102AE0006D917C918EE790E00E94960710921906F6
:102AF000DF91CF911F910F91FF90EF90DF90CF90DA
:102B0000BF90AF909F908F907F906F905F9008954F
:102B10002F923F924F925F926F927F928F929F92ED
:102B2000AF92BF92CF92DF92EF92FF920F931F93DB
:102B3000CF93DF93CDB7DEB728970FB6F894DEBFFB
:102B40000FBECDBF2C012AEC421A2EEF520AF20121
:102B5000F0801C01F9EC2F1AFEEF3F0AF101008111
:102B60009C01285C3E4F3A832983F901F081F88764
:102B70009C01275C3E4F3C832B83F901F081FD8350
:102B8000FC01E65CFE4FB081FC01E55CFE4FA081DC
:102B9000FC01E45CFE4F7081FC01E35CFE4F1081A0
:102BA000FC01E25CFE4F6081FC01E15CFE4F508164
:102BB000FC01E05CFE4FE080FC01EF5BFE4F4081DA
:102BC000EF2DE07821E030E0E03811F020E030E057
:102BD000F901F695FE2FEE27F795E795FF83EE8333
:102BE000E1E0F02FF078F03809F0E0E02E81F0E439
:102BF000EF9F200D1124E22F31E0212F2078203883
:102C000009F030E0E30F31E028852078203809F022
:102C100030E0F0E23F9FE00D112431E02D8120787B
:102C2000203809F030E020E1329FE00D112431E03E
:102C30002B2F2078203809F030E0F8E03F9FE00D9E
:102C4000112431E02A2F2078203809F030E024E0E8
:102C5000329FE00D112421E030E0F72FF078F038BA
:102C600011F020E030E0220F331F2E0FF2012083FD
:102C700021E030E0F6FC02C020E030E03695322F53
:102C8000222737952795E1E006FFE0E0522EF0E499
:102C9000EF9F500C1124E52D31E016FF30E0E30FDB
:102CA00031E0288526FF30E0F0E23F9FE00D11245F
:102CB00031E05D8056FE30E020E1329FE00D1124CE
:102CC00031E0B6FF30E0F8E03F9FE00D112431E045
:102CD000A6FF30E024E0329FE00D112421E030E037
:102CE00076FD02C020E030E0220F331F2E0FF101ED
:102CF000208321E030E0E62FE078E03811F020E09A
:102D000030E03695322F222737952795E1E0F52FD1
:102D1000F078F03809F0E0E0522EF0E4EF9F500C2C
:102D20001124E52D31E046FF30E0E30F31E02E2D98
:102D30002078203809F030E020E2329FE00D1124A5
:102D400031E0242F2078203809F030E0F0E13F9F77
:102D5000E00D112431E066FF30E028E0329FE00D05
:102D6000112431E056FF30E0F4E03F9FE00D1124E4
:102D700021E030E0E6FC02C020E030E0220F331F0B
:102D80002E0FE981FA81208321E030E0F5FC02C0BA
:102D900020E030E03695322F222737952795E1E065
:102DA00005FFE0E0522EF0E4EF9F500C1124E52DDA
:102DB00031E015FF30E0E30F31E0288525FF30E0FA
:102DC000F0E23F9FE00D112431E05D8055FE30E0E0
:102DD00020E1329FE00D112431E0B5FF30E0F8E052
:102DE0003F9FE00D112431E0A5FF30E024E0329F49
:102DF000E00D112421E030E075FD02C020E030E05C
:102E0000220F331F2E0FEB81FC812083FC01E65C37
:102E1000FE4F21E030E0F4FC02C020E030E0190178
:102E20003694322C2224379427945524539404FF4B
:102E3000512C322D20E4529E300D1124532E31E0BE
:102E400014FF30E0530E31E0288524FF30E020E20B
:102E5000329F500C112431E02D8124FF30E020E11D
:102E6000329F500C112431E0B4FF30E028E0329F53
:102E7000500C112431E0A4FF30E024E0329F500CCC
:102E8000112421E030E074FD02C020E030E0220F88
:102E9000331F250D2083FC01E55CFE4F21E030E06F
:102EA00065FD02C020E030E019013694322C222466
:102EB000379427945524539455FF512C222D30E4F8
:102EC000539E200D1124522E31E044FF30E0530E6A
:102ED00031E0E5FE30E020E2329F500C112431E079
:102EE00045FF30E020E1329F500C112431E064FFB7
:102EF00030E028E0329F500C112431E054FF30E0E4
:102F000024E0329F500C112421E030E0E4FC02C0A8
:102F100020E030E0220F331F250D2083FC01E45C0C
:102F2000FE4F21E030E0F3FC02C020E030E0190168
:102F30003694322C2224379427945524539403FF3B
:102F4000512C222D30E4539E200D1124522E31E0BD
:102F500013FF30E0530E31E0288523FF30E020E2FC
:102F6000329F500C112431E02D8123FF30E020E10D
:102F7000329F500C112431E0B3FF30E028E0329F43
:102F8000500C112431E0A3FF30E024E0329F500CBC
:102F9000112421E030E073FD02C020E030E0220F78
:102FA000331F250D2083FC01E35CFE4F21E030E060
:102FB000F2FC02C020E030E019013694322C2224C9
:102FC000379427945524539402FF512C222D30E43A
:102FD000539E200D1124522E31E012FF30E0530E8B
:102FE00031E0288522FF30E020E2329F500C11248E
:102FF00031E02D8122FF30E020E1329F500C11247E
:1030000031E0B2FF30E028E0329F500C112431E073
:10301000A2FF30E024E0329F500C112421E030E088
:1030200072FD02C020E030E0220F331F250D208307
:10303000FC01E25CFE4F21E030E063FD02C020E0D5
:1030400030E019013694322C2224379427945524E9
:10305000539453FF512C222D30E4539E200D112404
:10306000522E31E042FF30E0530E31E0E3FE30E01B
:1030700020E2329F500C112431E043FF30E020E188
:10308000329F500C112431E062FF30E028E0329F83
:10309000500C112431E052FF30E024E0329F500CFC
:1030A000112421E030E0E2FC02C020E030E0220FF9
:1030B000331F250D2083FC01E15CFE4F21E030E051
:1030C000F1FC02C020E030E019013694322C2224B9
:1030D000379427945524539401FF512C222D30E42A
:1030E000539E200D1124522E31E011FF30E0530E7B
:1030F00031E0288521FF30E020E2329F500C11247E
:1031000031E02D8121FF30E020E1329F500C11246D
:1031100031E0B1FF30E028E0329F500C112431E063
:10312000A1FF30E024E0329F500C112421E030E078
:1031300071FD02C020E030E0220F331F250D2083F7
:10314000FC01E05CFE4FF0FAFF24F0F800FBCC2419
:10315000C0F8D12C26E0CC0CDD1C2A95E1F730E834
:10316000F39EC01811241170C10E3885317020E211
:10317000329FC00C11243D81317020E1329FC00C80
:103180001124B17038E0B39FC00C1124A17024E069
:10319000A29FC00C112470FBAA24A0F8B12CAA0C89
:1031A000BB1CCA0CC082FC01EF5BFE4F262F2170B6
:1031B00050FB882480F8912C880C991C880C991C51
:1031C00038E0239F800C1124242F2170820EE0FA16
:1031D000662460F8712C660C771C860C21E061FF78
:1031E00020E080E8289F8018112421E051FF20E092
:1031F00030E4239F800C112421E0E1FE20E080E2F6
:10320000289F800C112421E041FF20E030E1239F22
:10321000800C1124808228960FB6F894DEBF0FBE72
:10322000CDBFDF91CF911F910F91FF90EF90DF9075
:10323000CF90BF90AF909F908F907F906F905F9056
:103240004F903F902F9008952F923F924F925F9210
:103250006F927F928F929F92AF92BF92CF92DF92A6
:10326000EF92FF920F931F93CF93DF93CDB7DEB70B
:103270002F970FB6F894DEBF0FBECDBF8C019C0117
:103280002C5E3E4F3E832D839C012F5D3E4F3A873F
:1032900029872C0131EE431A3EEF530A7C0140EEA0
:1032A000E41A4EEFF40A6C0188EEC81A8EEFD80AC1
:1032B00018019BED291A9EEF390AAD81BE818D91CF
:1032C0009C910E94CC079C018F3FBFEF9B0709F4A4
:1032D0009EC14FB7F8948091140690911506A09165
:1032E0001606B09117064FBFE985FA858083918352
:1032F000A283B383D2014C91442309F4E6C02B315D
:10330000310529F4F7018081882309F4DEC0D60154
:103310008D919C91119701968D939C936CE070E038
:103320000E94482C892B09F0D0C02B31310529F09F
:10333000C9018E579109029710F4F70110825801C4
:10334000FAEEAF1AFEEFBF0AD5016D917C91C8016C
:1033500041E050E0FC01E60FF71F3B97A081FC0124
:10336000EA5CFE4FA0834F5F5F4F01964C305105E2
:1033700089F7F801EF5BFE4F2083C8010E94881592
:10338000F50180809180F3E08F1A9108D5018D922C
:103390009C925801612C712C9801265E3E4F3C870F
:1033A0002B879801235E3E4F38872F83F501EA5C17
:1033B000FE4F2081F501E95CFE4F3081F501E85CAC
:1033C000FE4F9081632F822F2D873E879F870E941B
:1033D0002C0EAB85BC858C939F8589272D853E85DA
:1033E000882309F44EC0982F9F70998382958F701F
:1033F0008A83FE01319680E090E041915FEF540FA7
:103400005230D0F14430C1F14830B1F14330E9F0ED
:10341000453009F435C1463041F0473071F049304C
:1034200071F050E04A3069F002C054E00FC04B30F8
:1034300051F04C3059F450E809C058E007C050E151
:1034400005C050E203C050E401C051E08130910555
:1034500009F014C12527442379F0D1014D915D91E4
:103460006D917C9113974F5F5F4F6F4F7F4F4D93DF
:103470005D936D937C93139701968230910509F0CB
:10348000BCCF822F8327EF81F885908189278083A5
:10349000C30163E070E00E945C2C660F771F680D2B
:1034A000791D600F711FFB0138972083FB0137974F
:1034B0003083F3E06F0E711C23E0A20EB11C3CE0E0
:1034C0006316710409F072CFF8CED7018C91811187
:1034D00084C02E37310509F073C0F60180819181D7
:1034E00098012A5E3E4F4901D801A35EBE4F5D019F
:1034F0000C9708F452C02FB7F8948091140690915D
:103500001506A0911606B09117062FBFE985FA851A
:1035100080839183A283B383D5018C9181113DC0B7
:10352000D8018D91982F92959F70282F217080FF40
:1035300002C0A90FB11DF40160817181625071094F
:10354000929F6019710911247C836B8381FD04C0F3
:10355000F80120E030E00CC0CD010E94F40F9C8304
:103560008B83AC0168E075E0C8010E94372E08C06B
:103570002617370729F08D9181932F5F3F4FF8CFA2
:103580001A830983F801E55EFE4F0190F081E02D7A
:10359000309719F0CE010196099581E0D2018C9304
:1035A000F40111821082D6011D921C928AEAF50163
:1035B0008083D1011D921D921D921C9213977DCE86
:1035C0002F37310519F4F201108277CE2B313105F6
:1035D00021F481E0D7018C9370CE4423A9F0F80147
:1035E000EA5EFE4F808191818431B1E09B0750F407
:1035F000AC014F5F5F4F51834083F801E80FF91F23
:10360000208302C0F2011082D7011C9256CEED81B8
:10361000FE8100811181D8011C968D919C911D978E
:10362000892B41F449E451E06DE273E083E293E0D9
:103630000E94E229D8011C96ED91FC911D97C801CA
:103640000995892BF9F0ED81FE8100811181D80166
:103650001E968D919C911F97892B41F442E551E074
:1036600061E173E084E093E00E94E229D8011E96B4
:10367000ED91FC911F97C801099504C03527EBCE49
:1036800052E0E4CE2F960FB6F894DEBF0FBECDBF4A
:10369000DF91CF911F910F91FF90EF90DF90CF902E
:1036A000BF90AF909F908F907F906F905F904F9062
:1036B0003F902F900895CF93FC01603208F04EC0E8
:1036C0008081918170E0892B79F4268530E0AB010F
:1036D0004150510981E090E002C0880F991F4A953E
:1036E000E2F728173907D4F120E030E0C0E82617C8
:1036F00037076CF58685811118C08081918100970C
:1037000069F1A281B381AD014F5F5F4F5383428363
:10371000AE0FBF1F5396AC91A5874817590721F4E8
:103720001382128211821082C68782859385880F48
:10373000991F9387828756854585452319F08160B7
:1037400093878287569556872F5F3F4FD0CF6285EC
:1037500073851386128680E090E003C06FEF7FEFE1
:10376000CB01CF9108950C944A2DCF93DF93EC01B8
:1037700041E050E00F8402C0440F551F0A94E2F765
:1037800089899A89480F591F60E070E0CE014396FD
:103790000E94522E1C86198218821B821A821E8653
:1037A0001D861D821C821F821E82198618861B861A
:1037B0001A86DF91CF910895EF92FF920F931F9396
:1037C000CF93DF9300D0CDB7DEB78C018CEF860F9F
:1037D0008C3030F50115110519F1423008F16417EC
:1037E000F8F081E090E0062E02C0880F991F0A943D
:1037F000E2F798012D5E3F4F820F931F4A83698342
:103800000E94B22C7C014A816981009749F0FC0139
:10381000128B018B6787408B0E94B51BC70102C0CA
:1038200080E090E00F900F90DF91CF911F910F916A
:10383000FF90EF900895EF92FF920F931F93CF9315
:10384000DF93EC017901009789F16115710571F140
:103850002115310559F188819981E989FA89E81B97
:10386000F90B31F4F9011182108281E090E020C05F
:103870008A01E417F50708F48F014396A8018C0F1D
:103880009D1F0E94372E88819981800F911F9983F7
:1038900088838C85811104C081E08C871B821A8209
:1038A000F7011183008380E090E002C08FEF9FEF6B
:1038B000DF91CF911F910F91FF90EF9008952F927C
:1038C0003F925F927F928F929F92AF92BF92CF92E0
:1038D000DF92EF92FF920F931F93CF93DF93EC0150
:1038E0007B016A018901009709F427C161157105FF
:1038F00009F423C12115310509F41FC1D9011D9215
:103900001C92AA24A394B12C7C84872D90E089304A
:10391000910508F014C1FC01EC5CFF4F0C94922C53
:1039200080E090E00EC161E0CE010E945B1B672B3E
:10393000682B692B69F48F85893008F04CC01F8291
:103940001E8266C0F801808191818C159D0510F062
:1039500082E0DDC068E0CE010E945B1B6F3FFFEF9D
:103960007F078F079F07A1F3E989FA897396EC0F08
:10397000FD1FD5010F8402C0AA0FBB1F0A94E2F7F6
:10398000119728853985A9014F5F5F4F598748876F
:10399000A223B323EA0FFB1F6083D8014D915C91F2
:1039A00011979A012F5F3F4F2D933C93F701E40F3E
:1039B000F51F6083A9C06F856850CE010E945B1B14
:1039C0006F3FBFEF7B078B079B0729F0762F66279A
:1039D0007F836E831DC083E09AC06F85693008F0D5
:1039E00068E0CE010E945B1B6F3FEFEF7E078E0702
:1039F0009E0771F02E813F81262B372B2F5F3F4F83
:103A00003F832E8388891D821C82893058F112C021
:103A100084E07DC068896850CE010E945B1B6F3FC7
:103A2000FFEF7F078F079F0729F0762F66277D839B
:103A30006C8318C085E06BC06889693008F068E065
:103A4000CE010E945B1B6F3F2FEF72078207920728
:103A500049F02C813D81262B372B2F5F3F4F3D8333
:103A60002C8354C086E053C0D8018D919C91B6013F
:103A7000681B790B09F44AC08C819D8186179707D2
:103A800008F4BC0189899A8943968C0F9D1FA50172
:103A90000F8402C0440F551F0A94E2F741505109A8
:103AA0008E809F8020E030E02617370729F1E885D7
:103AB000F985E819F909E423F523E80FF91F508087
:103AC000D801ED91FC911F01BFEF2B1A3B0AD801E1
:103AD0002D923C92EE0DFF1D5082E885F985E4237E
:103AE000F523E80FF91F5082E885F9853196F987AB
:103AF000E8872F5F3F4FD8CF8C819D81821B930B2E
:103B00009D838C83892B11F488E001C087E08C872A
:103B100007C021E088819981892B09F420E02C8756
:103B20008C858711F1CE81E090E0F8012081318110
:103B30002C153D0531F080E004C08FEF01C08EEF01
:103B40009FEFDF91CF911F910F91FF90EF90DF904A
:103B5000CF90BF90AF909F908F907F905F903F905D
:103B60002F900895FC01009789F08485882321F027
:103B70008350843070F402C080E00CC081E090E09B
:103B800020813181232B39F480E008958FEF9FEF5E
:103B9000089581E090E008958F929F92BF92CF9216
:103BA000DF92EF92FF920F931F93CF93DF93EC017D
:103BB000E62EF42E890188E0861748F443E452E0AB
:103BC0006AE473E08FE393E00E94E22917C0A8E063
:103BD0006A1314C08E85803889F4E901E881F9817F
:103BE000AC81BD818D919C9111979C012F5F3F4FBE
:103BF0002D933C93E80FF91F408342C080E090E092
:103C00006E2D70E06150710988248394912C4F2DA2
:103C100050E030E8B32E9B01281B390B2F3FBFEF3C
:103C20003B0771F1F40102C0EE0FFF1F2A95E2F786
:103C30009F0124233523EE85232B19F02D852E2B70
:103C40002D872E2F269511F02E8718C0BE86D801FD
:103C5000ED91FC9111971496ED90FC901597D7017A
:103C60002D913C916901BFEFCB1ADB0AD701CD92B0
:103C7000DC92FD84E20FF31FF0821D860196CBCF0C
:103C8000DF91CF911F910F91FF90EF90DF90CF9038
:103C9000BF909F908F9008951F93CF93DF93EC0177
:103CA0009B011A85193050F018504885598502C07B
:103CB000569547951A95E2F718E003C048851123F9
:103CC00039F0612FCE010E94CC1D8A85811B8A8725
:103CD000812FDF91CF911F9108950C944A2DCF939E
:103CE000DF93EC0142E050E00F8402C0440F551F07
:103CF0000A94E2F760E070E041960E94522E198229
:103D000018821C861B821A821B8680E88E871D867D
:103D10001D821C82198618861A86DF91CF9108951C
:103D2000EF92FF921F93CF93DF931F92CDB7DEB731
:103D3000182F8CEF810F8C30D8F46230C8F0161732
:103D4000B8F082E090E0012E02C0880F991F0A941B
:103D5000E2F7419669830E94B22C7C016981009749
:103D600039F0FC011787608B0E946F1EC70102C0EB
:103D700080E090E00F90DF91CF911F91FF90EF9046
:103D80000895CF92DF92EF92FF920F931F93CF93FC
:103D9000DF93EC0169010097A9F16115710591F1BB
:103DA0002115310579F18B8580FD2FC08C8581111E
:103DB0002CC081E090E00F8402C0880F991F0A9404
:103DC000E2F7288139817C01E21AF30A87014E1556
:103DD0005F0508F48A01820F931F4196A8018C0F9A
:103DE0009D1F0E94372EF6011183008388819981DF
:103DF000800F911F998388830E151F0549F481E078
:103E00008C8706C08FEF9FEF05C08EEF9FEF02C03B
:103E100080E090E0DF91CF911F910F91FF90EF90A4
:103E2000DF90CF9008952F923F924F925F926F92C2
:103E30007F928F929F92AF92BF92CF92DF92EF923A
:103E4000FF920F931F93CF93DF93CDB7DEB76297A7
:103E50000FB6F894DEBF0FBECDBF8C013A01490109
:103E6000009709F4E8C16115710509F4E4C1211551
:103E7000310509F4E0C14115510509F4DFC1D9014B
:103E80001D921C927A8369835C834B833E832D83CE
:103E9000EE24E394F12C1C01B1E12B0E311CF8014E
:103EA000F485F88B8F2F90E08A30910508F0C6C119
:103EB000FC01E35CFF4F0C94922CE2E0D8011C96CD
:103EC000EC93A9C1D8011F96EC911F97570150960A
:103ED0000C90509702C0AA0CBB1C0A94E2F71296F1
:103EE0004D915C9113971B966C911B978D919C91B2
:103EF00060FF03C020E030E001C09501DC01A21B9F
:103F0000B30B4A175B0708F08AC0970102C0220F63
:103F1000331FEA95E2F7F9012901440E551E64FFAB
:103F200003C0FA0131960AC063FF08C09A012F5FEF
:103F30003F4FF501A216B30608F4F901841B950B57
:103F40008A159B0508F45C01B101640D751D7D8720
:103F50006C87B201615071098FEF8F83CC24CA94B2
:103F60001A8A198A6E177F0794F19B018C859D85AB
:103F70009B878A87D101A60FB71FB987A88780E0E2
:103F800090E08A159B0571F0A885B985DD90B98709
:103F9000A887DE86AA85BB85DD90BB87AA87AE850C
:103FA000AD1549F0A989BA89A817B90730F02F8152
:103FB0003C2DCD0105C00196E4CF8A159B0559F033
:103FC000615071092F83C32E9A8B898BCBCF2F81A0
:103FD0003C2D89899A898330910540F0F201E21BDA
:103FE000F30B9F012F3FFFEF3F0799F44F5F5F4FA8
:103FF000D80113965C934E9312971B968C911B9746
:1040000082601B968C931B9715961C921E92149798
:10401000AFC0F8013783268395838483A9C087E0E6
:10402000D3C0ED81FE81208131818B819C81281755
:10403000390728F5F801848195819E012F5F3F4F54
:10404000892B39F441E061E0C8010E94CC1D84E075
:1040500017C040E061E0C8010E94CC1DD80116964F
:104060008D919C911797019719969C938E93189711
:104070001F968C911F971A968C9385E001C083E060
:10408000F8018487C8C0ED81FE81208131818B8158
:104090009C812817390730F5C701D8011F960C906D
:1040A0001F9702C0880F991F0A94E2F71296ED91AC
:1040B000FC911397E00FF11FE80FF91F9E012F5F8E
:1040C0003F4F408968E0C8010E94CC1DF8018385FC
:1040D000982F9D7F938782FD76C084819581892B5F
:1040E000E9F146C084E070C0ED81FE81208131811C
:1040F0008B819C812817390710F085E065C0BE01CF
:104100006F5F7F4FC8010E944C1E8111F6CFF801EE
:10411000848195810197918780878089828709C0F2
:10412000ED81FE81208131818B819C8128173907A7
:1041300010F086E049C0BE016F5F7F4FC8010E944A
:104140004C1E8111F6CFF801828193812481358143
:10415000820F931F938382831582148282E034C07E
:10416000F801838580FF06C081FF2DC084608387AE
:1041700083E02AC0A701078402C0440F551F0A9498
:10418000E2F7A280B380440F551F4A195B09B501BD
:104190006F5E7F4F600F711FC1010E94402EF801BA
:1041A000838583FF03C08061838702C08860838723
:1041B000F80113821282808191818A199B0991836F
:1041C000808380E001C088E0D8011C968C9323C0D6
:1041D000F80186858038B9F0AD81BE818D919C91C2
:1041E00011972B813C818217930778F4E981FA813A
:1041F0009C012F5F3F4F2D933C93D8011D962C912E
:10420000E80FF91F208389E001C088E0F801848766
:1042100080E090E015C0D8011C968C91D8888D1153
:104220003ECED4018D919C918615970509F037CE2D
:1042300081E090E005C08FEF9FEF02C08EEF9FEF0F
:1042400062960FB6F894DEBF0FBECDBFDF91CF915F
:104250001F910F91FF90EF90DF90CF90BF90AF90A4
:104260009F908F907F906F905F904F903F902F9096
:104270000895FC01009779F08385816083878485A8
:10428000811102C081E0848781E090E0248529309B
:1042900021F480E008958FEF9FEF08952F923F92D1
:1042A0004F925F926F927F928F929F92AF92BF9246
:1042B000CF92DF92EF92FF920F931F93CF93DF93F2
:1042C000CDB7DEB7C45AD1090FB6F894DEBF0FBE22
:1042D000CDBFC856DF4F99838883C859D040C65692
:1042E000DF4F79836883CA59D040C456DF4F598362
:1042F0004883CC59D0405901C257DF4F19821882E8
:10430000CE58D0409E012F5F3F4FC957DF4F3983B2
:104310002883C758D040AE014A575F4FC757DF4F79
:1043200059834883C958D040C856DF4F0881198146
:10433000C859D0400F5F1F4FC856DF4FE881F98141
:10434000C859D0408491853291F1882309F448C737
:10435000C456DF4F68817981CC59D040C656DF4FB3
:10436000E881F981CA59D0400995C257DF4FE880EA
:10437000F980CE58D040FFEFEF1AFF0AC557DF4F44
:10438000B982A882CB58D040C856DF4F1983088322
:10439000C859D040C257DF4FF982E882CE58D0408A
:1043A000C557DF4FA880B980CB58D040BDCFF801AA
:1043B0008491853259F5C856DF4F28813981C85913
:1043C000D0402E5F3F4FC856DF4F39832883C859EE
:1043D000D040C456DF4F68817981CC59D040C65651
:1043E000DF4FE881F981CA59D0400995C257DF4FA4
:1043F000E880F980CE58D040FFEFEF1AFF0AC5578A
:10440000DF4FB982A882CB58D040C4CFC256DF4F0D
:104410001882CE59D040C357DF4F1882CD58D040B4
:10442000C057DF4F1882C059D040CF56DF4F188297
:10443000C159D040F8012491C80101962B3209F4EA
:1044400058C060F42032E9F0233209F05AC0F1E09C
:10445000C357DF4FF883CD58D04051C02D3251F0B3
:10446000203309F04EC021E0C256DF4F2883CE59D9
:10447000D04045C0F1E0C057DF4FF883C059D0406D
:104480003EC0232D2C7F322ECF56DF4F3881C159AD
:10449000D040332ACE56DF4F4881C259D04040FB2E
:1044A00032F8C057DF4F5881C059D04050FB33F825
:1044B00020FA34F8CD56DF4FA881C359D040A0FB75
:1044C00035F8C357DF4FB881CD58D040B0FB36F830
:1044D000CC56DF4FE881C459D040E0FB37F8232D9C
:1044E000237069F441E0CF56DF4F4883C159D04073
:1044F00006C031E0CF56DF4F3883C159D0408C0120
:1045000099CFC357DF4F5881CD58D040C056DF4FA9
:104510005883C05AD040F80124912A3221F0612CEE
:10452000712C3AE025C095012E5F3F4FD5016D906B
:104530007C9077FE09C0719461947108B1E0C05716
:10454000DF4FB883C059D0408C01590116C02A33BF
:10455000A0F40F5F1F4FFC018491A301349F300131
:10456000359F700C112450E3651A7108680E711C98
:10457000C801F8012491203350F7C057DF4FF8816C
:10458000C059D040FF2329F0C256DF4F1882CE59C0
:10459000D040F80184918E3249F5319684918A3267
:1045A00029F08F01412C512C3AE01AC0D5014D90D1
:1045B0005C900E5F1F4FF50132965F011AC02A33DF
:1045C000C0F40F5F1F4FFC018491A201349F2001B2
:1045D000359F500C112450E3451A5108480E511CC8
:1045E000C801F8012491203350F703C044244A94B1
:1045F000542CF8012491C8010196283699F018F43A
:104600002C3439F017C02C3621F02A3799F4212C9C
:1046100002C0222423948C01CD56DF4F1882C35947
:10462000D0400EC08C01F1E0CD56DF4FF883C35966
:10463000D04005C0CD56DF4F1882C359D040212C41
:1046400098012F5F3F4FC856DF4F39832883C859E1
:10465000D040F801D490C956DF4FD882C759D04016
:10466000F5E6DF1609F402C2FD15ECF023E5D216DB
:1046700009F453C02D1564F035E4D31609F4F6C1DE
:1046800047E4D41609F4E1C1DD2009F46FC42AC05F
:1046900053E6D51671F15D150CF4C6C088E5D81641
:1046A00009F48DC01FC090E7D91609F471C09D159B
:1046B00064F0A7E6DA1609F4C8C1DA160CF4D1C121
:1046C000B9E6DB1609F4B0C00DC0E5E7DE1609F463
:1046D00076C0F8E7DF1609F46DC023E7D21202C0F6
:1046E000F12C1DC0C557DF4FB982A882CB58D040EE
:1046F00049C4A5014E5F5F4FC557DF4F59834883BB
:10470000CB58D040D5018C918983F12C8E010E5F5E
:104710001F4FFE0131964F0143C4FF24F3949501CE
:104720002E5F3F4FC557DF4F39832883CB58D0408A
:10473000D5018D909C908114910421F4A4E28A2EDD
:10474000A1E09A2E57FE04C0F0E14F2EF7E25F2E53
:104750008401FF20C1F0F8018491882309F420C46A
:10476000C80188199909841595050CF019C40F5FC3
:104770001F4FF1CFC80188199909841595050CF0D0
:104780000FC40F5F1F4FD8018C918111F3CF08C464
:10479000F5013296C557DF4FF983E883CB58D040F7
:1047A000D5016D917C9180E090E0E3E4EE2EE1E0B4
:1047B000FE2E26C073E5E72E71E0F72E04C063E4F9
:1047C000E62E61E0F62E222071F0F5013496C557F1
:1047D000DF4FF983E883CB58D040D5016D917D91AF
:1047E0008D919C910DC0C5010296F501608171818A
:1047F000C557DF4F99838883CB58D04080E090E045
:1048000021E0CE56DF4F2883C259D04035E7D3127E
:1048100005C0CE56DF4F1882C259D040CF56DF4F69
:104820001882C159D0403EC0222079F0A5014C5FCA
:104830005F4FC557DF4F59834883CB58D040D501D0
:104840006D917D918D919C910FC0F5013296C55768
:10485000DF4FF983E883CB58D040D5016D917C912F
:10486000882777FD8095982F97FF13C090958095A6
:10487000709561957F4F8F4F9F4FCE56DF4F1882B7
:10488000C259D040B2E0CF56DF4FB883C159D040B3
:1048900005C0CE56DF4F1882C259D04053E4E52EF2
:1048A00051E0F52EE1E0CC56DF4FE883C459D0400B
:1048B000611571058105910529F4CC56DF4F1882E9
:1048C000C459D0404114510441F4CC56DF4FF88113
:1048D000C459D040FF2309F476C0CE56DF4F28815B
:1048E000C259D0408E010A571F4F2130A9F02AE04B
:1048F00030E040E050E00E94702CF701E60FF71F17
:104900008081D8018E938D01B901CA0161157105AD
:104910008105910561F715C0FB01EF70FF27EE0DD2
:10492000FF1D2081F80122938F0144E09695879521
:10493000779567954A95D1F76115710581059105C0
:1049400059F757FE43C0C256DF4FF881CE59D040C9
:10495000FF23E1F1232D2C7F322ECF56DF4F3881FC
:10496000C159D040332ACE56DF4F4881C259D0407A
:1049700040FB32F8C057DF4F5881C059D04050FB40
:1049800033F820FA34F8CD56DF4F8881C359D04030
:1049900080FB35F8C357DF4F9881CD58D04090FB4E
:1049A00036F8CC56DF4FA881C459D040A0FB37F869
:1049B000232D237081E090E011F480E090E023014A
:1049C000481A590A03C08E010A571F4FC757DF4FB5
:1049D00088819981C958D040801B910BF80120E350
:1049E0004F01841595051CF422930196F9CFC35706
:1049F000DF4FB881CD58D040BB23A1F0CC56DF4F5C
:104A0000E881C459D040EE2369F08D2D8F7D883523
:104A100049F4F4013197D082F2E08F1A910880E3D3
:104A2000D4018C93C957DF4FE881F981C758D04032
:104A30008E169F0608F0AEC247EB52E064E873E0C2
:104A400081E793E00E94E229A5C2DA94DA94C9567C
:104A5000DF4FD882C759D04011E04114510469F0AA
:104A600006C0C956DF4F1882C759D04010E057FE24
:104A700007C026E0422E512C03C044244394512CFD
:104A800095012C5F3F4FC557DF4F39832883CB58A3
:104A9000D040D501CD90DD90ED90FC9020E030E04D
:104AA000A901C701B6010E94822A87FF0AC0F7FA4E
:104AB000F094F7F8F094B2E0CF56DF4FB883C159C5
:104AC000D040C156DF4F1883CF59D04088248394FB
:104AD000912C8C0E9D1E860C971C20E030E040E847
:104AE0005FE3C701B6010E94D12B87FD32C0A12C24
:104AF000B12C27EB33E44AEB51E5C701B6010E9424
:104B0000D12B87FD0EC029EF32E045E150E5C7010A
:104B1000B6010E94862A6B017C01EAE0AE0EB11C50
:104B2000E8CF20E030E040E251E4C701B6010E9446
:104B3000D12B87FD49C020E030E040E251E4C701BD
:104B4000B6010E94862A6B017C01FFEFAF1ABF0AF3
:104B5000E8CF20E030E0A901C701B6010E94822A17
:104B6000A12CB12C882381F12FEF36EE4BED5EE2C4
:104B7000C701B6010E94822A181674F029EF32E0AC
:104B800045E150E5C701B6010E94D52B6B017C01C0
:104B90002AE0A21AB108E8CF20E030E040E85FE365
:104BA000C701B6010E94822A87FF0EC020E030E0D4
:104BB00040E251E4C701B6010E94D52B6B017C0194
:104BC00031E0A31AB108E8CF112321F1A414B504F0
:104BD00064F44CEFA4164FEFB4063CF04A185B089F
:104BE000C956DF4F1882C759D04051E0451A5108C5
:104BF00081E0C357DF4F9881CD58D0409827C156E8
:104C0000DF4F9883CF59D040A1E0C357DF4FA8832F
:104C1000CD58D040C956DF4FB881C759D040B111E7
:104C20004CC0B7FE3EC080E3E1E0F0E0EC0FFD1FBA
:104C3000E60DF71D80834114510461F4C357DF4F23
:104C4000E881CD58D040E11105C0F401319680E0F3
:104C500090E007C0F40132968EE2D40111968C9355
:104C6000C20195012F5F3F4F280F391F40E38F018D
:104C70008217930729F0009719F041930197F7CF16
:104C8000920120953095A216B3060CF4D6C02C01E3
:104C9000E1E0F0E0CB56DF4FF983E883C559D0401F
:104CA0005CC0222733272A193B09CB56DF4F3983B3
:104CB0002883C559D040840150C08401CB56DF4FB2
:104CC00019821882C559D04048C0C701B6010E9458
:104CD000EE2ACF55DF4F688379838A839B83C15A3D
:104CE000D040CF55DF4F48815981C15AD040BA01D9
:104CF000882777FD8095982F0E94212B9B01AC017E
:104D0000C701B6010E941D2A20E030E040E251E4D4
:104D10000E94D52B6B017C0198012F5F3F4FCF552F
:104D2000DF4F8881C15AD040805DD8018C93CB562B
:104D3000DF4F88819981C559D0400196CB56DF4F0E
:104D4000E881F981C559D040EF2B91F0CB56DF4F68
:104D500099838883C559D0408901CB56DF4F28817C
:104D60003981C559D040421653060CF0AECF14C05D
:104D70004114510439F4C357DF4FF881CD58D04066
:104D8000FF2339F098012E5F3F4FEEE2D8011196D4
:104D9000EC9381E090E0DACF20E030E040EA50E4AC
:104DA000C701B6010E94D12B87FD47C0F80181E001
:104DB00090E030E322912E3251F0820F8A3321F0BD
:104DC000808380E090E003C0308381E090E08E1625
:104DD0009F0680F3892B89F1C956DF4F3881C75967
:104DE000D0403323B9F0F8018E169F0678F4DF0126
:104DF0008E919D018E3239F4CF010297DC018C91A6
:104E00008083F90101C080833197EECFBFEFAB1AE9
:104E1000BB0A0BC00F5F1F4FF8018E169F0628F4C8
:104E2000DF018E918083FD01F8CF81E3E1E0F0E0C6
:104E3000EC0FFD1FE60DF71D8083C156DF4FE881A3
:104E4000CF59D040EE2349F0F8018291803311F41C
:104E50008F01FACF8E3209F48F01C956DF4FF881E6
:104E6000C759D040FF23B9F1D801FC93C80102967D
:104E7000B7FE07C02DE211962C93B194A194B1080E
:104E800004C02BE2D80111962C938C01065F1F4FB2
:104E900020E030E02F5F3F4FF8013196C5016AE016
:104EA00070E00E945C2C805DD8018C935B016115E1
:104EB000710511F08F01EECF22303105DCF3E21BDA
:104EC000F30B199781918E93215031091216130615
:104ED000CCF309501109C256DF4FB881CE59D040EA
:104EE000BB2309F45CC0E32DEC7F3E2ECF56DF4F91
:104EF000F881C159D0403F2ACE56DF4F2881C25990
:104F0000D04020FB32F8C057DF4F3881C059D04025
:104F100030FB33F820FA34F8CD56DF4F4881C359BF
:104F2000D04040FB35F8C056DF4F5881C05AD040C2
:104F300050FB36F8CC56DF4F8881C459D04080FBF7
:104F400037F8232D237081E090E011F480E090E0A9
:104F50009301281B390BF40140E34F01C8018E1B5C
:104F60009F0B82179307DCF44293F7CFC557DF4FAF
:104F7000B982A882CB58D040C856DF4F1983088326
:104F8000C859D040F12C03E211E080E2882E81E084
:104F9000982E06C0F12C8E010A571F4F01C0F12C2C
:104FA0000819190960167106DCF1932D9C7F392EC2
:104FB000CF56DF4FA881C159D0403A2ACE56DF4F95
:104FC000B881C259D040B0FB32F8C057DF4FE881FA
:104FD000C059D040E0FB33F820FA34F8CD56DF4F0B
:104FE000F881C359D040F0FB35F8C056DF4F288117
:104FF000C05AD04020FB36F8CC56DF4F3881C45918
:10500000D04030FB37F86301C01AD10A232D23703A
:1050100081E090E011F480E090E0C81AD90A02C063
:10502000C12CD12CC057DF4F4881C059D04041110D
:1050300022C031E0C31AD108D7FC1DC0C456DF4FCF
:1050400068817981CC59D04080E2C656DF4FE88133
:10505000F981CA59D0400995C257DF4F288139815B
:10506000CE58D0402F5F3F4FC257DF4F3983288340
:10507000CE58D040DECF432D4C7F342ECF56DF4F5D
:105080005881C159D040352ACE56DF4F8881C25948
:10509000D04080FB32F8C057DF4F9881C059D040D4
:1050A00090FB33F820FA34F8CD56DF4FA881C3596E
:1050B000D040A0FB35F8C056DF4FB881C05AD04071
:1050C000B0FB36F8CC56DF4FE881C459D040E0FB46
:1050D00037F8832D837001F1813011F48BE201C028
:1050E0008DE2C456DF4F68817981CC59D040C656D5
:1050F000DF4FE881F981CA59D0400995C257DF4F87
:1051000028813981CE58D0402F5F3F4FC257DF4FA3
:1051100039832883CE58D040F11009C0C257DF4FE1
:10512000A880B980CE58D040A818B90822C0C2576C
:10513000DF4FE880F980CE58D0405401AE18BF0848
:105140000150110917FD2DC0F501EE0DFF1D8491D1
:10515000C456DF4F68817981CC59D040C656DF4FA5
:10516000E881F981CA59D0400995FFEFEF1AFF0A8B
:10517000E7CF7501E80CF91C0150110917FD11C0AA
:10518000C456DF4F68817981CC59D040D4018D91CC
:105190004D01C656DF4FE881F981CA59D0400995C3
:1051A000E8CFC057DF4FF881C059D040FF2309F442
:1051B000F1C821E0C21AD108D7FCECC8C456DF4FB1
:1051C00068817981CC59D04080E2C656DF4FE881B2
:1051D000F981CA59D0400995FFEFEF1AFF0AE9CFCC
:1051E000C257DF4F88819981CE58D040CC55DF4FD0
:1051F0000FB6F894DEBF0FBECDBFDF91CF911F91E8
:105200000F91FF90EF90DF90CF90BF90AF909F9065
:105210008F907F906F905F904F903F902F90089568
:105220009091C00095FFFCCF8A3041F09091C00072
:1052300090649093C0008093C60008959091C00040
:1052400090649093C0009DE09093C6009091C00040
:1052500095FFFCCFEBCFCF939B01C091C100409154
:10526000C10048604093C1004091C1004F79409314
:10527000C10040E050E060E179E20E944E2180915F
:10528000C00086FFFCCFC093C100CF910895CF939B
:10529000C091C1009091C10098609093C10090911D
:1052A000C1009F799093C10060E070E00E941029D6
:1052B0008091C00086FFFCCFC093C100CF910895BC
:1052C000CF93DF93CDB7DEB7FE01359681919191F3
:1052D000BF010E942B29DF91CF9108951F93CF9397
:1052E000DF931091C1002091C10028602093C1007C
:1052F0002091C1002F792093C100FC018491EF011E
:105300002196882331F060E070E00E941029FE01B0
:10531000F5CF8091C00086FFFCCF1093C100DF91D4
:10532000CF911F910895AF92BF92CF92DF92EF92EB
:10533000FF920F931F93CF93DF936C0185E0E82ECC
:10534000F12C00E117E2C0E0D0E09AE0A92EB12CE8
:10535000C601B8010E945C2C6C016115710529F42D
:10536000209719F40130110529F480E3860F0E947B
:1053700047292196C801B5010E945C2C8B0181E070
:10538000E81AF108E114F10419F7CE01DF91CF9189
:105390001F910F91FF90EF90DF90CF90BF90AF9053
:1053A0000895CF93DF93EB010E946E298AE30E9458
:1053B0004729CE010E94932983EB93E0DF91CF919F
:1053C0000C946E29CF93DF93EC01CB01BA010E94BC
:1053D000D12986EB93E00E946E29CE010E946E29AE
:1053E0008AE00E94472981E090E0DF91CF91089503
:1053F0000F931F93CF93DF93182F092FEB01B90160
:10540000CA010E94D12985EA93E00E946E29CE014B
:105410000E946E290F931F938CE993E09F938F93C3
:105420000E9460290F900F900F900F9081E090E004
:10543000DF91CF911F910F9108955058BB27AA2754
:105440000ED075C166D130F06BD120F031F49F3FA2
:1054500011F41EF45BC10EF4E095E7FB51C1E92F96
:1054600077D180F3BA17620773078407950718F09E
:1054700071F49EF58FC10EF4E0950B2EBA2FA02D7E
:105480000B01B90190010C01CA01A0011124FF27F1
:10549000591B99F0593F50F4503E68F11A16F040EC
:1054A000A22F232F342F4427585FF3CF46953795EB
:1054B0002795A795F0405395C9F77EF41F16BA0BB0
:1054C000620B730B840BBAF09150A1F0FF0FBB1F5E
:1054D000661F771F881FC2F70EC0BA0F621F731FA7
:1054E000841F48F4879577956795B795F7959E3F04
:1054F00008F0B3CF9395880F08F09927EE0F979592
:1055000087950895D9D008F481E008950CD00FC193
:1055100007D140F0FED030F021F45F3F19F0F0C029
:10552000511139C1F3C014D198F39923C9F355230C
:10553000B1F3951B550BBB27AA2762177307840786
:1055400038F09F5F5F4F220F331F441FAA1FA9F33C
:1055500033D00E2E3AF0E0E830D091505040E6952E
:10556000001CCAF729D0FE2F27D0660F771F881F8F
:10557000BB1F261737074807AB07B0E809F0BB0B7E
:10558000802DBF01FF2793585F4F2AF09E3F5105A2
:1055900068F0B6C000C15F3FECF3983EDCF386953F
:1055A00077956795B795F7959F5FC9F7880F911D18
:1055B0009695879597F90895E1E0660F771F881F04
:1055C000BB1F621773078407BA0720F0621B730BB7
:1055D000840BBA0BEE1F88F7E095089504D0689409
:1055E000B111D9C00895BCD088F09F5790F0B92F61
:1055F0009927B751A0F0D1F0660F771F881F991F28
:105600001AF0BA95C9F712C0B13081F0C3D0B1E039
:105610000895C0C0672F782F8827B85F39F0B93F49
:10562000CCF3869577956795B395D9F73EF4909529
:105630008095709561957F4F8F4F9F4F0895E894A7
:1056400009C097FB3EF490958095709561957F4FCA
:105650008F4F9F4F9923A9F0F92F96E9BB27939578
:10566000F695879577956795B795F111F8CFFAF488
:10567000BB0F11F460FF1BC06F5F7F4F8F4F9F4FB9
:1056800016C0882311F096E911C0772321F09EE817
:10569000872F762F05C0662371F096E8862F70E07D
:1056A00060E02AF09A95660F771F881FDAF7880F57
:1056B0009695879597F90895990F0008550FAA0BAD
:1056C000E0E8FEEF16161706E807F907C0F0121615
:1056D0001306E407F50798F0621B730B840B950B18
:1056E00039F40A2661F0232B242B252B21F408956D
:1056F0000A2609F4A140A6958FEF811D811D08950A
:1057000097F99F6780E870E060E008959FEF80EC74
:10571000089500240A941616170618060906089517
:1057200000240A9412161306140605060895092E7D
:105730000394000C11F4882352F0BB0F40F4BF2BEC
:1057400011F460FF04C06F5F7F4F8F4F9F4F08952C
:1057500057FD9058440F551F59F05F3F71F0479522
:10576000880F97FB991F61F09F3F79F08795089507
:10577000121613061406551FF2CF4695F1DF08C026
:10578000161617061806991FF1CF86957105610543
:1057900008940895E894BB2766277727CB0197F9EB
:1057A00008958ADF08F48FEF08950BD0C0CFB1DFE2
:1057B00028F0B6DF18F0952309F0A2CFA7CF112467
:1057C000EACFC6DFA0F3959FD1F3950F50E0551FA8
:1057D000629FF001729FBB27F00DB11D639FAA2746
:1057E000F00DB11DAA1F649F6627B00DA11D661F95
:1057F000829F2227B00DA11D621F739FB00DA11DB6
:10580000621F839FA00D611D221F749F3327A00D6F
:10581000611D231F849F600D211D822F762F6A2F0B
:1058200011249F5750408AF0E1F088234AF0EE0F90
:10583000FF1FBB1F661F771F881F91505040A9F79D
:105840009E3F510570F05CCFA6CF5F3FECF3983ED2
:10585000DCF3869577956795B795F795E7959F5F04
:10586000C1F7FE2B880F911D9695879597F908959E
:10587000DB018F939F930E94982CBF91AF91A29FC1
:10588000800D911DA39F900DB29F900D112408953E
:10589000AA1BBB1B51E107C0AA1FBB1FA617B70756
:1058A00010F0A61BB70B881F991F5A95A9F7809572
:1058B0009095BC01CD01089597FB072E16F4009436
:1058C00007D077FD09D00E94482C07FC05D03EF494
:1058D000909581959F4F0895709561957F4F08959C
:1058E000A1E21A2EAA1BBB1BFD010DC0AA1FBB1FE4
:1058F000EE1FFF1FA217B307E407F50720F0A21B56
:10590000B30BE40BF50B661F771F881F991F1A94C2
:1059100069F760957095809590959B01AC01BD01EC
:10592000CF010895EE0FFF1F0590F491E02D09942B
:105930000E94A32CA59F900DB49F900DA49F800D55
:10594000911D11240895A29FB001B39FC001A39F90
:10595000700D811D1124911DB29F700D811D1124A8
:10596000911D0895CF93DF938230910510F482E06A
:1059700090E0E0911D06F0911E0620E030E0A0E0EE
:10598000B0E0309739F14081518148175907B8F09C
:105990004817590771F482819381109729F0139663
:1059A0009C938E9312972CC090931E0680931D0695
:1059B00027C02115310531F04217530718F0A9010E
:1059C000DB0101C0EF019A01BD01DF010280F3811B
:1059D000E02DD7CF21153105F9F0281B390B2430E4
:1059E000310580F48A819B816115710521F0FB01ED
:1059F0009383828304C090931E0680931D06FE014C
:105A0000329644C0FE01E20FF31F8193919322501E
:105A10003109398328833AC020911B0630911C0636
:105A2000232B41F4209102013091030130931C0695
:105A300020931B06209100013091010121153105B1
:105A400041F42DB73EB74091040150910501241B4C
:105A5000350BE0911B06F0911C06E217F307A0F44A
:105A60002E1B3F0B2817390778F0AC014E5F5F4FB4
:105A70002417350748F04E0F5F1F50931C064093C4
:105A80001B068193919302C0E0E0F0E0CF01DF912B
:105A9000CF910895CF93DF93009709F487C0FC015D
:105AA000329713821282C0911D06D0911E06209754
:105AB00081F420813181280F391F80911B0690913C
:105AC0001C068217930779F5F0931C06E0931B06DA
:105AD0006DC0DE0120E030E0AE17BF0750F4129633
:105AE0004D915C9113979D014115510509F1DA0122
:105AF000F3CFB383A28340815181840F951F8A170E
:105B00009B0771F48D919C911197840F951F0296BC
:105B10009183808312968D919C91139793838283B6
:105B20002115310529F4F0931E06E0931D063EC0B1
:105B3000D9011396FC93EE9312974D915D91A40FAA
:105B4000B51FEA17FB0779F480819181840F951FB7
:105B50000296D90111969C938E938281938113961C
:105B60009C938E931297E0E0F0E08A819B810097EE
:105B700019F0FE01EC01F9CFCE010296288139819E
:105B8000820F931F20911B0630911C06281739079E
:105B900069F4309729F410921E0610921D0602C077
:105BA00013821282D0931C06C0931B06DF91CF9103
:105BB00008958F929F92AF92BF92CF92DF92EF9211
:105BC000FF92CF93DF93EC01688179818A819B8179
:105BD000611571058105910521F464E279ED8BE58C
:105BE00097E02DE133EF41E050E00E94612E490142
:105BF0005A019B01AC01A7EAB1E40E94982C6B0109
:105C00007C01ACEEB4EFA50194010E945C2EC60E9F
:105C1000D71EE81EF91EF7FE06C081E0C81AD1089B
:105C2000E10880E8F80AC882D982EA82FB82C601CC
:105C30009F77DF91CF91FF90EF90DF90CF90BF9053
:105C4000AF909F908F9008950E94D92D089586E07F
:105C500091E00E94D92D0895A0E0B0E08093060164
:105C600090930701A0930801B09309010895FB01E7
:105C7000DC0102C001900D9241505040D8F70895C8
:105C80006817790768F4FB01DC01E40FF51FA40F26
:105C9000B51F02C002900E9241505040D8F70895AF
:105CA0000C94372EDC0101C06D9341505040E0F759
:105CB0000895B7FF0C94982C0E94982C821B930B8C
:105CC0000895052E97FB1EF400940E94782E57FD30
:105CD00007D00E94702C07FC03D04EF40C94782E51
:105CE00050954095309521953F4F4F4F5F4F089508
:105CF00090958095709561957F4F8F4F9F4F089538
:045D0000F894FFCF45
:105D040000001F0620000100000037018401640127
:105D140020002000002B0164016401000000000049
:105D24003F3F3F003C4E554C4C3E0023023A02425A
:105D34000243024702440204020A02710217020DDE
:105D44000244023031323334353637383941424334
:105D5400444546303132333435363738396162633D
:045D6400646566000C
:00000001FF
